:100000000EC028C027C026C025C02BC023C022C0D8
:1000100021C020C01FC01EC01DC01CC01BC0112499
:100020001FBECFE5D2E0DEBFCDBF10E0A0E6B0E05E
:10003000E8E4F1E002C005900D92A036B107D9F7CF
:1000400010E0A0E6B0E001C01D92A936B107E1F7CB
:1000500004D078C0D5CF0895089557D0FCDFFCDFD9
:10006000FECF1F920F920FB60F9211242F933F9342
:100070004F935F936F937F938F939F93AF93BF93B0
:1000800020916400309165004091660050916700B6
:1000900070916800DA01C9014096A11DB11D672F5A
:1000A000605D6D3730F06D57DA01C9014196A11DD1
:1000B000B11D609368008093640090936500A093E5
:1000C0006600B09367008091600090916100A091FC
:1000D0006200B09163000196A11DB11D8093600084
:1000E00090936100A0936200B0936300BF91AF91C1
:1000F0009F918F917F916F915F914F913F912F9140
:100100000F900FBE0F901F90189578948AB582605B
:100110008ABD8AB581608ABD83B7826083BF83B799
:10012000816083BF89B7826089BF80B7826080BFEA
:1001300080B7816080BF80B7806480BF319A309A79
:08014000379A0895F894FFCFEF
:00000001FF
